:020000040000FA
:10000000003083168600850083122D200A201520DB
:1000100021200928103084001030A3002308562026
:100020008000840AA30B0E28080080303620083098
:10003000A2001F308400000842208403A20B1B286A
:100040000800C03036200830A200173084000008B5
:1000500042208403A20B27280800383036200130C4
:100060003620033036200F303620080086004E2020
:10007000043085004E20003085004E20043085007D
:100080004E20080086004E20063085004E200230AB
:1000900085004E20063085004E2008006430A10007
:1000A000A000A00B5128A10B502808008207203483
:1000B00020344534443455345034493443342034A6
:1000C0002034313436344634383434342034203417
:02400E00F13F80
:00000001FF
